:100000000C942A000C9445000C9445000C94450077
:100010000C9445000C9445000C9445000C9445004C
:100020000C9445000C9445000C9445000C9445003C
:100030000C9445000C9445000C9445000C9445002C
:100040000C9445000C9445000C9445000C9445001C
:100050000C94450011241FBECFE5D4E0DEBFCDBF18
:1000600010E0A0E6B0E0E8E2F7E002C005900D92F3
:10007000A036B107D9F710E0A0E6B0E001C01D92AC
:10008000A036B107E1F70C9459030C940000CF930C
:10009000DF93CDB7DEB724970FB6F894DEBF0FBE5F
:1000A000CDBF19821A821B821C8289819A81AB8101
:1000B000BC8186309105A105B10560F489819A81E2
:1000C000AB81BC810196A11DB11D89839A83AB834D
:1000D000BC83EBCF24960FB6F894DEBF0FBECDBF26
:1000E000DF91CF910895CF93DF93CDB7DEB72697F9
:1000F0000FB6F894DEBF0FBECDBF89839A831B82F3
:100100001C821D821E8289819A819C01442737FDB1
:100110004095542F8B819C81AD81BE812817390772
:100120004A075B07E0F089819A819C01442737FDEB
:100130004095542F8B819C81AD81BE812817390752
:100140004A075B0700F38B819C81AD81BE810196DC
:10015000A11DB11D8B839C83AD83BE83E4CF269606
:100160000FB6F894DEBF0FBECDBFDF91CF910895DB
:10017000CF93DF93CDB7DEB723970FB6F894DEBFEA
:100180000FBECDBF898388E090E08A839B838A81FC
:100190009B81181619067CF58A819B8101978A83B9
:1001A0009B838981882394F48091320082608093BC
:1001B0003200809132008160809332000E944700BB
:1001C000809132008E7F8093320011C08091320086
:1001D0008D7F809332008091320081608093320065
:1001E0000E944700809132008E7F80933200898187
:1001F000880F8983CCCF23960FB6F894DEBF0FBE4D
:10020000CDBFDF91CF910895CF93DF93CDB7DEB708
:1002100023970FB6F894DEBF0FBECDBF88E090E005
:1002200089839A831B8289819A81181619062CF575
:100230008B81880F8B8380913200816080933200A4
:10024000809130009927969587959695879581702E
:100250009070009721F08B8181608B8303C08B812C
:100260008E7F8B8389819A81019789839A8380917C
:1002700032008E7F80933200D6CF8B81992787FD05
:10028000909523960FB6F894DEBF0FBECDBFDF91D9
:10029000CF910895CF93DF93CDB7DEB722970FB6F6
:1002A000F894DEBF0FBECDBF898380913200877F77
:1002B000809332009FE789818923898389810E9405
:1002C000B8000E9447000E9404018A838A8199270E
:1002D00022960FB6F894DEBF0FBECDBFDF91CF914F
:1002E0000895CF93DF93CDB7DEB722970FB6F8947A
:1002F000DEBF0FBECDBF89836A8380913200877FC6
:100300008093320090E88981892B898389810E94BA
:10031000B8008A810E94B800809132008860809382
:10032000320022960FB6F894DEBF0FBECDBFDF912C
:10033000CF910895CF93DF93CDB7DEB78BE3809352
:100340003100809132008B7F809332008FEF809359
:1003500037008FEF80933800DF91CF910895CF93CE
:10036000DF93CDB7DEB78091320080618093320099
:1003700080E197E20E947300809132008F7E80932B
:100380003200DF91CF910895CF93DF93CDB7DEB7E1
:100390008091320088608093320080E991E00E9471
:1003A000730080913200877F80933200DF91CF917C
:1003B0000895CF93DF93CDB7DEB78091320080628E
:1003C000809332000E9447000E9447000E94AF01C4
:1003D0000E94C401DF91CF9108950F931F93CF9393
:1003E000DF93CDB7DEB724970FB6F894DEBF0FBE0C
:1003F000CDBF89839A836B837C8382E00E944A010C
:1004000088237CF409811A8183E00E944A01F80163
:1004100080830B811C8184E00E944A01F801808363
:1004200006C0E981FA811082EB81FC81108224965A
:100430000FB6F894DEBF0FBECDBFDF91CF911F91F5
:100440000F910895CF93DF93CDB7DEB722970FB604
:10045000F894DEBF0FBECDBF82E00E944A01882320
:100460000CF583E00E944A01833050F083E00E9443
:100470004A018D3F28F481E090E089839A8314C07B
:1004800084E00E944A01833050F084E00E944A01D7
:100490008D3F28F481E090E089839A8305C019821A
:1004A0001A8202C019821A8289819A8122960FB615
:1004B000F894DEBF0FBECDBFDF91CF910895CF93EB
:1004C000DF93CDB7DEB722970FB6F894DEBF0FBE2D
:1004D000CDBF85E00E944A01863028F081E090E09F
:1004E00089839A8302C019821A8289819A8122960D
:1004F0000FB6F894DEBF0FBECDBFDF91CF91089548
:10050000CF93DF93CDB7DEB72C970FB6F894DEBF4D
:100510000FBECDBF89839A836B837C8382E00E9468
:100520004A0188230CF0BCC083E00E944A0199274D
:10053000AA27BB278D839E83AF83B88784E00E9460
:100540004A019927AA27BB2789879A87AB87BC8747
:100550008D819E81AF81B88583309105A105B1055C
:100560000CF44AC08D819E81AF81B8858D3F910585
:10057000A105B1050CF040C08D819E81AF81B88589
:1005800080389105A105B105CCF069817A81E981B6
:10059000FA8120813181428153818D819E81AF8199
:1005A000B885820F931FA41FB51F80509140A040B3
:1005B000B040FB0180839183A283B3838D819E81B0
:1005C000AF81B8858F379105A105B105ACF469817C
:1005D0007A81E981FA8120813181428153818D8143
:1005E0009E81AF81B885820F931FA41FB51FFB01A9
:1005F00080839183A283B38389859A85AB85BC85EB
:1006000083309105A105B1050CF44AC089859A850E
:10061000AB85BC858D3F9105A105B1050CF040C0AF
:1006200089859A85AB85BC8580389105A105B10582
:10063000CCF06B817C81EB81FC8120813181428116
:10064000538189859A85AB85BC85820F931FA41F32
:10065000B51F80509140A040B040FB018083918342
:10066000A283B38389859A85AB85BC858F37910535
:10067000A105B105ACF46B817C81EB81FC8120810B
:100680003181428153818D819E81AF81B885820FF6
:10069000931FA41FB51FFB0180839183A283B383A3
:1006A0002C960FB6F894DEBF0FBECDBFDF91CF9171
:1006B0000895C4E5D4E0DEBFCDBF0E949A018091C9
:1006C00032008860809332000E94D9011B821C8214
:1006D0001D821E821F82188619861A868FEF8093CC
:1006E0003400109235001B866B858AE00E947101F0
:1006F000CE0107969E012D5F3F4FBC01C9010E94AC
:1007000080028B819C81AD81BE8180959095A09562
:10071000B095892F9A2FAB2FBB27A7FDBA95809351
:0807200038000E944700E4CFFD
:00000001FF
